:1000000003EF16F0000000004FEF15F000000000B5
:0C0010000000000000000000D3EF15F01D
:0C001C0072B201D0FDD75FC573FF120067
:0E002800ACB202D00000FCD75FC5ADFF1200E5
:10003600C7B409D01F0EC514016E0150000A03E1B2
:0A004600010E006E01D0006A1200E6
:100050006DB409D01F0E6B14016E0150000A03E14C
:0A006000010E006E01D0006A1200CC
:10006A00F250026EF29E0500FF6A0150FE6E0050C9
:08007A00FD6E02BEF28E1200C1
:0A008200000E9EBA010E006E12007F
:10008C0074CF01F071A202D07198718801C000F098
:02009C00120050
:0A009E00000EACB2010E006E12005D
:1000A8004DC05BF54EC05CF54FC05DF550C05EF5C8
:1000B8000501596B5A6B5A51120802E159518E08C1
:1000C80008E3B5DF005201E004D00501594B5A2B73
:1000D800F2D70501120E5A5D02E18F0E595D03E356
:1000E8007B0E006E24D0C580C5A020D04D504E1088
:1000F8004F1050101AE05B515C115D115E110EE15A
:1001080074C3E1FF75C3E2FF050EE66E72C300F02B
:1001180073C301F0A6DF010E006E09D0010E0501C0
:100128005B5F000E5C5B5D5B5E5BDED7006A1200A6
:0A013800000E72B2010E006E1200FC
:1001420051C05BF552C05CF553C05DF554C05EF51D
:100152000501596B5A6B5A51120802E159518E0826
:1001620008E375DF005201E004D00501594B5A2B18
:10017200F2D70501120E5A5D02E18F0E595D03E3BB
:100182007B0E006E24D06B806BA020D05150521099
:10019200531054101AE05B515C115D115E110EE1B7
:1001A20078C3E1FF79C3E2FF050EE66E76C300F085
:1001B20077C301F059DF010E006E09D0010E05016F
:1001C2005B5F000E5C5B5D5B5E5BDED7006A12000C
:1001D200AECF01F0ABA202D0AB98AB8801C000F069
:0201E200120009
:0A01E400000EA4BA010E006E120016
:0C01EE00B8C300F0B9C301F039DF120003
:1001FA0053C504F00000000000000000026A036A10
:10020A00800E0318006E800E005C02E1080E025C8C
:10021A001FE2800E0414016E0150800A02E18B8AEB
:10022A0001D08B9A020E0D6E0D2EFED700000436F9
:10023A0004908B86020E0D6E0D2EFED700008B9653
:10024A00020E0D6E0D2EFED70000024A032AD8D7E1
:02025A00120090
:10025C0051C053F552C054F553C055F554C056F522
:10026C006B826BA21FD0515052105310541019E0D6
:10027C00050153515411551156110CE178C3E1FF8E
:10028C0079C3E2FF060EE66E76C300F077C301F089
:10029C00E6DE08D0010E0501535F000E545B555B82
:0602AC00565BDFD71200D3
:1002B200A49E53C56FFF51C054F552C055F553C0AB
:1002C20056F554C057F56DA421D051505210531019
:1002D20054101BE0050154515511561157110EE1EE
:1002E20078C3E1FF79C3E2FF040EE66E76C300F045
:1002F20077C301F0B9DE010E006E3AD0010E05019E
:10030200545F000E555B565B575BDDD751C054F509
:1003120052C055F553C056F554C057F5A4BE21D06E
:1003220051505210531054101BE0050154515511F5
:10033200561157110EE178C3E1FF79C3E2FF040EB3
:10034200E66E76C300F077C301F08EDE010E006E1A
:100352000FD0010E0501545F000E555B565B575BD3
:10036200DDD76BBC02D0006A03D06B84020E006E34
:02037200120077
:040374006B84120084
:1003780051C055F552C056F553C057F554C058F5FD
:10038800A49E6B86A4BE1FD0515052105310541017
:1003980019E0050155515611571158110CE178C350
:1003A800E1FF79C3E2FF030EE66E76C300F077C380
:1003B80001F057DE08D0010E0501555F000E565BAF
:1003C800575B585BDFD705016FCF54F55351000ACF
:1003D80002E16B8A01D06B9AA49E6B8851C055F5D7
:1003E80052C056F553C057F554C058F5A4BE1FD097
:1003F800515052105310541019E00501555156111F
:10040800571158110CE178C3E1FF79C3E2FF030EDD
:10041800E66E76C300F077C301F023DE08D0010E44
:100428000501555F000E565B575B585BDFD754C517
:0404380000F01200BE
:10043C000B6A0A6A096A086A0E6A033408360450A1
:10044C00085E0550D8A0053C095E0650D8A0063CB5
:10045C000A5E0750D8A0073C0B5EE86AD8A0010ED4
:10046C000E5E0336070E0C6E0334083609360A3658
:10047C000B360E36045003A012D0085E0550D8A0DF
:10048C00053C095E0650D8A0063C0A5E0750D8A071
:10049C00073C0B5EE86AD8A0010E0E5E11D0082650
:1004AC000550D8B0053C09260650D8B0063C0A26A3
:1004BC000750D8B0073C0B26E86AD8B0010E0E26C0
:1004CC0003360C2ED1D70234083609360A360B36D1
:1004DC000E36045003A012D0085E0550D8A0053C7F
:1004EC00095E0650D8A0063C0A5E0750D8A0073C0F
:1004FC000B5EE86AD8A0010E0E5E11D008260550DE
:10050C00D8B0053C09260650D8B0063C0A26075040
:10051C00D8B0073C0B26E86AD8B0010E0E2602367E
:10052C00070E0C6E0234083609360A360B360E36B8
:10053C00045002A012D0085E0550D8A0053C095EFC
:10054C000650D8A0063C0A5E0750D8A0073C0B5EAC
:10055C00E86AD8A0010E0E5E11D008260550D8B05E
:10056C00053C09260650D8B0063C0A260750D8B0E0
:10057C00073C0B26E86AD8B0010E0E2602360C2E6C
:10058C00D1D70134083609360A360B360E360450EC
:10059C0002A012D0085E0550D8A0053C095E06509A
:1005AC00D8A0063C0A5E0750D8A0073C0B5EE86A50
:1005BC00D8A0010E0E5E11D008260550D8B0053C0F
:1005CC0009260650D8B0063C0A260750D8B0073C7E
:1005DC000B26E86AD8B0010E0E260136070E0C6EFB
:1005EC000134083609360A360B360E36045001A093
:1005FC0012D0085E0550D8A0053C095E0650D8A064
:10060C00063C0A5E0750D8A0073C0B5EE86AD8A0EF
:10061C00010E0E5E11D008260550D8B0053C0926F7
:10062C000650D8B0063C0A260750D8B0073C0B261B
:10063C00E86AD8B0010E0E2601360C2ED1D7003444
:10064C00083609360A360B360E36045001A012D085
:10065C00085E0550D8A0053C095E0650D8A0063CA3
:10066C000A5E0750D8A0073C0B5EE86AD8A0010EC2
:10067C000E5E11D008260550D8B0053C0926065050
:10068C00D8B0063C0A260750D8B0073C0B26E86ABF
:10069C00D8B0010E0E260036070E0C6E003408364C
:1006AC0009360A360B360E36045000A012D0085EFE
:1006BC000550D8A0053C095E0650D8A0063C0A5E41
:1006CC000750D8A0073C0B5EE86AD8A0010E0E5E5E
:1006DC0011D008260550D8B0053C09260650D8B0D4
:1006EC00063C0A260750D8B0073C0B26E86AD8B05F
:1006FC00010E0E2600360C2ED1D700B00ED00450B1
:10070C0008260550D8B0053C09260650D8B0063C42
:0C071C000A260750D8B0073C0B2612003C
:100728000CDDD00E0501536FC0DD4AC553F5BDDDA4
:1007380004DDD10E0501536FB8DD0501536B18DEDA
:1007480000C0D9F3000E0301DA6F10DED9C300F040
:0207580012008D
:10075A0049DDD00E0501536FA7DD4AC553F5A4DD67
:10076A004BC553F5A1DD75DD05014C6B4D6B800E54
:10077A004D19006E800E005C02E1030E4C5D0DE225
:10078A00D00E536F91DD0050010A02E1D5DC01D091
:0E079A0004D005014C4B4D2BEAD7E7DD1200D1
:1007A80005014A51390806E3300E4A5D03E3010E9C
:0807B800006E01D0006A12007E
:1007C0008B90060E0D6E0D2EFED700004AC553F518
:1007D00014DD4BC553F511DD4AC553F50EDD4CC58F
:1007E00053F50BDD4AC553F508DD4DC553F505DD61
:1007F0004AC553F502DD4EC553F5FFDC4AC553F536
:10080000FCDC4FC553F5F9DC4AC553F5F6DC50C5A1
:1008100053F5F3DC4AC553F5F0DC51C553F5EDDC77
:100820004AC553F5EADC52C553F5E7DC060E0D6EFA
:0A0830000D2EFED700008B80120091
:10083A000B6A0A6A096A00500402F4CF09F0F3CF7E
:10084A0008F001500502F4CF0BF0F3CF0AF0005084
:10085A000502F3500926F4500A22E86A0B220150D5
:10086A000402F3500926F4500A22E86A0B2208C04F
:10087A0000F009C001F00AC002F00BC003F0120038
:10088A000450085E0550D8A0053C095E0650D8A061
:10089A00063C0A5E0750D8A0073C0B5E0336070EDB
:1008AA000C6E0334083609360A360B36045003A098
:1008BA000ED0085E0550D8A0053C095E0650D8A0A7
:1008CA00063C0A5E0750D8A0073C0B5E0DD00826EE
:1008DA000550D8B0053C09260650D8B0063C0A2671
:1008EA000750D8B0073C0B2603360C2EDAD7023451
:1008FA00083609360A360B36045003A00ED0085EB5
:10090A000550D8A0053C095E0650D8A0063C0A5EF0
:10091A000750D8A0073C0B5E0DD008260550D8B06A
:10092A00053C09260650D8B0063C0A260750D8B01E
:10093A00073C0B260236070E0C6E023408360936BF
:10094A000A360B36045002A00ED0085E0550D8A015
:10095A00053C095E0650D8A0063C0A5E0750D8A09E
:10096A00073C0B5E0DD008260550D8B0053C092679
:10097A000650D8B0063C0A260750D8B0073C0B26CA
:10098A0002360C2EDAD70134083609360A360B3607
:10099A00045002A00ED0085E0550D8A0053C095E9E
:1009AA000650D8A0063C0A5E0750D8A0073C0B5E4A
:1009BA000DD008260550D8B0053C09260650D8B0F7
:1009CA00063C0A260750D8B0073C0B260136070E0C
:1009DA000C6E0134083609360A360B36045001A06B
:1009EA000ED0085E0550D8A0053C095E0650D8A076
:1009FA00063C0A5E0750D8A0073C0B5E0DD00826BD
:100A0A000550D8B0053C09260650D8B0063C0A263F
:100A1A000750D8B0073C0B2601360C2EDAD7003423
:100A2A00083609360A360B36045001A00ED0085E85
:100A3A000550D8A0053C095E0650D8A0063C0A5EBF
:100A4A000750D8A0073C0B5E0DD008260550D8B039
:100A5A00053C09260650D8B0063C0A260750D8B0ED
:100A6A00073C0B260036070E0C6E00340836093692
:100A7A000A360B36045000A00ED0085E0550D8A0E6
:100A8A00053C095E0650D8A0063C0A5E0750D8A06D
:100A9A00073C0B5E0DD008260550D8B0053C092648
:100AAA000650D8B0063C0A260750D8B0073C0B2699
:100ABA0000360C2EDAD700B00ED0045008260550A6
:100ACA00D8B0053C09260650D8B0063C0A2607507D
:080ADA00D8B0073C0B26120006
:100AE200086A080E0C6E003408360450085ED8B04E
:0E0AF20002D00826D89000360C2EF5D7120040
:100B00000B1E0A1E091E081E082AD8B4092AD8B4CA
:080B10000A2AD8B40B2A1200D6
:100B18003CC5F6FF3DC5F7FF3EC5F8FF0900F5CF18
:100B280000F0005212E03CC5F6FF3DC5F7FF3EC598
:100B3800F8FF0900F5CF5FF514EC00F0010E050190
:0C0B48003C27000E3D233E23E3D71200A3
:100B54000D0E05015F6F14EC00F00A0E05015F6FC6
:060B640014EC00F0120089
:100B6A0005013C6B060E3C5D0FE23C51010F4A6FDA
:100B7A004B6B4C6B4D6B4E6B4F6B506B516B526B9F
:0A0B8A001ADE05013C2BEED7120025
:100B9400A69C3DC5AAFF3CC5A9FFA69EA680A8CFDA
:040BA40000F012004B
:060BA80000000000120035
:100BAE00086A096A100E0C6E0134083609360450B4
:100BBE00085E0550D8A0053C095ED8B007D0045099
:100BCE0008260550D8B0053C0926D89000360136C7
:060BDE000C2EEAD7120004
:100BE4000301CA51CB1101E015D005014A6B9ADD0E
:100BF4007F0E0014D96FDA6B000EDA17000EDA6F6D
:100C040005014A6BD9C34BF5A6DD010E0301CA6F7A
:060C1400000ECB6F120080
:100C1A00030E006E3CC543F5000E0501446F0050FB
:100C2A0005E0433743914437FF0FFAD7456B320E3D
:100C3A003C25F66E420EF76E000EF722000EF86E95
:100C4A00000EF8220900F5CFEAF0416B426B000E64
:100C5A00425D02E1080E415DD8B0D3D03F0E3F6F2E
:100C6A00000E406F000E006E4051005C02E13F51E1
:100C7A00000819E2EA0E3F25E16E000E4021E26EFD
:100C8A00010E3F5D006E000E4059016EEA0E00240F
:100C9A00E96E000E0120EA6EEECFE6FF010E3F5F1D
:100CAA00000E405BDFD743514125006E445142217B
:100CBA00016E320E0024F66E420E0120F76E000E0F
:100CCA00F86E000EF8220900F5CFEAF0456B080E1F
:100CDA003F6F000E406F000E006E4051005C02E153
:100CEA003F51000876E23FC54AF5EA0EE96E000E6A
:100CFA00EA6E4551E926D8B0EA2AEECF4BF5080E3E
:100D0A004525006E016A000E0122EA0E0024E96EF2
:100D1A00000E0120EA6EEECF4CF5100E4525006E4E
:100D2A00016A000E0122EA0E0024E96E000E01207B
:100D3A00EA6EEECF4DF5180E4525006E016A000EDB
:100D4A000122EA0E0024E96E000E0120EA6EEECFBF
:100D5A004EF5200E4525006E016A000E0122EA0EAC
:100D6A000024E96E000E0120EA6EEECF4FF5280E40
:100D7A004525006E016A000E0122EA0E0024E96E82
:100D8A00000E0120EA6EEECF50F5300E4525006EBA
:100D9A00016A000E0122EA0E0024E96E000E01200B
:100DAA00EA6EEECF51F5380E4525006E016A000E47
:100DBA000122EA0E0024E96E000E0120EA6EEECF4F
:100DCA0052F5F9DC0501452B010E3F5F000E405B31
:100DDA0082D73F6B406B3E51405D02E13D513F5D22
:100DEA000DE2030E0C6E970E0D6E0D2EFED70C2E15
:100DFA00FCD7000000003F4B402BEDD7414B422B64
:040E0A0026D71200D5
:100E0E0005014A6B8ADC800E0010D96FDA6B000E7A
:100E1E00DA13000EDA6F05014A6BD9C34BF596DC77
:080E2E000301CA6BCB6B12003B
:100E36000501426B436B000E435D02E10A0E425D03
:100E46000BE242514025E16E43514121E26E200EF4
:100E5600E66E424B432BEFD742514025E16E43519C
:100E66004121E26EE66A010E425F000E435B42518B
:100E76004025446F43514121456F0A0E046E000E12
:100E8600056E066E076E3CC500F03DC501F03EC519
:100E960002F03FC503F01EEC02F008C000F009C0E6
:100EA60001F00AC002F00BC003F0300E002644C564
:100EB600E1FF45C5E2FF00C0E6FF0A0E046E000E24
:100EC600056E066E076E3CC500F03DC501F03EC5D9
:100ED60002F03FC503F01EEC02F000C03CF501C075
:100EE6003DF502C03EF503C03FF5000E046E031843
:100EF60008E10450021805E10450011802E100500F
:100F0600000A01E105D0010E425F000E435BAFD738
:020F16001200C7
:100F180005013F6B3CC5E9FF3DC5EAFFEECF3EF555
:100F28003E51000A0FE03EC55FF514EC00F00501E4
:100F38003F2B3F513C25E96E000E3D21EA6EEECF76
:060F48003EF5EED7120099
:100F4E0040C500F005014007005228E03CC5E9FF0E
:100F5E003DC5EAFFEE50000A0CE03CC5E9FF3DC579
:100F6E00EAFF3EC5D9FF3FC5DAFFEE50DE1801E1BC
:100F7E000FD03CC5E9FF3DC5EAFF3EC5D9FF3FC5D1
:100F8E00DAFFDE50EE5C006E016A000E015A08D0E8
:100F9E0005013C4B3D2B3E4B3F2BD2D7006A016ADD
:020FAE0012002F
:100FB000A1EC00F0D00E0501536F59EC01F00501D2
:100FC000536B59EC01F0800E05013C25006E000EBC
:100FD0003D21016E00C053F559EC01F03EC553F5BB
:100FE00059EC01F040C553F559EC01F042C553F5F9
:100FF00059EC01F044C553F559EC01F046C553F5E1
:1010000059EC01F048C553F559EC01F0BAEC01F088
:10101000A1EC00F01A0E0C6EF80E0D6E0D2EFED720
:101020000C2EFCD70000D00E0501536F59EC01F0D7
:101030000501536B59EC01F00501536B59EC01F0BC
:06104000BAEC01F0120001
:101046003CC502F03DC503F002C000F003C001F04C
:10105600024A032A00C0E9FF01C0EAFFEE5201E09E
:10106600F3D705013C51025C006E3D510358016EF9
:0A107600010E005E000E015A120088
:1010800005013E6B3F6B3CC503F03DC504F03CC51C
:1010900005F03DC506F003C0E9FF04C0EAFFEE50CD
:1010A000200A04E13E513F1101E110D0010E3E6FD4
:1010B000000E3F6F03C0E9FF04C0EAFF05C0E1FF77
:1010C00006C0E2FFEECFE6FF054A062A03C001F0A4
:1010D00004C002F0034A042A01C0E9FF02C0EAFF8B
:1010E000EE50000AD8E13CC500F03DC501F0120009
:1010F0008B90060E0D6E0D2EFED700003CC553F5ED
:10110000FDEC00F03DC553F5FDEC00F03CC553F59A
:10111000FDEC00F03EC553F5FDEC00F03CC553F589
:10112000FDEC00F03FC553F5FDEC00F03CC553F578
:10113000FDEC00F040C553F5FDEC00F03CC553F567
:10114000FDEC00F041C553F5FDEC00F03CC553F556
:10115000FDEC00F042C553F5FDEC00F03CC553F545
:10116000FDEC00F043C553F5FDEC00F03CC553F534
:10117000FDEC00F044C553F5FDEC00F0060E0D6EDD
:0A1180000D2EFED700008B80120038
:10118A00020E0C6E490E0D6E0D2EFED70C2EFCD7DC
:06119A000000000012003D
:1011A0003CC5E9FF3DC5EAFFEE5005013E1905E1EA
:1011B0003CC500F03DC501F010D03CC500F03DC578
:1011C00001F03C4B3D2B00C0E9FF01C0EAFFEECF30
:0C11D00000F00052E5E1006A016A120024
:0A11DC00210E0D6E0D2EFED712003D
:0E11E600330E0D6E0D2EFED70000000012001D
:1011F400220E0C6E086A096A0A6A0B6A0C06D8B4D5
:101204001FD0D8900B320A3209320832033202322C
:1012140001320032D8A0F2D70C06D8B409D0045059
:1012240008260550092206500A2207500B22EAD745
:10123400045008260550092206500A2207500B22A2
:02124400120096
:101246000450000A12E10550000A0FE10650000A98
:101256000CE10750000A09E1FF0E006EFF0E016E59
:10126600FF0E026E7F0E036E99D00C6A07BE0C2A23
:101276000D6A0B6A0A6A096A086A035002100110AD
:101286000010D8B485D0035007180E6E0EBE0D1E82
:1012960007AE0BD0041E051E061E071E042AD8B470
:1012A600052AD8B4062AD8B4072A03AE0BD0001EE6
:1012B600011E021E031E002AD8B4012AD8B4022A2F
:1012C600D8B4032A035007100E6E0EBE1DD045EC8F
:1012D60004F00CBE36D00DAE5BD0001E011E021E01
:1012E600031E002AD8B4012AD8B4022AD8B4032A85
:1012F600081E091E0A1E0B1E082AD8B4092AD8B4CD
:101306000A2AD8B40B2A44D007AE15D003BE0DD096
:1013160003500B6E02500A6E0150096E0050086EA3
:10132600036A026A016A006AD6D7036A026A016A18
:10133600006A002A000C031E021E011E001E0C8EEF
:10134600C6D7082AD8B4092AD8B40A2AD8B40B2A88
:101356000450085CD8A4BFD70550095CD8A4BBD7F5
:1013660006500A5CD8A4B7D707500B5CD8A4B3D7ED
:101376000B6A0A6A096A086A002AD8B4012AD8B42C
:10138600022AD8B4032A03AEA6D70E6A0E88FF0C2B
:0E1396000E6A0CA002D080EC05F0000F1200D1
:1013A4003CC5E9FF3DC5EAFFEECF3EF5000E050161
:1013B4003F6F000E3F6F000E3F1902E1200E3E19F1
:1013C40007E0000E3F1902E1090E3E1901E003D0C7
:1013D4003C4B3D2BE5D7406B416B426B436B000E9E
:1013E4003F1902E12D0E3E1905E1424B432B3C4BC4
:1013F4003D2B08D0000E3F1902E12B0E3E1902E1ED
:101404003C4B3D2B3CC5E9FF3DC5EAFFEECF3EF525
:10141400000E3F6F000E3F6F3EC54AF5D4EC03F05B
:10142400005219E040C500F041C501F00A0E046EF7
:10143400000E056E1DEC04F0300E3E5D026E000ED3
:101444003F59036E02500024406F03500120416F46
:101454003C4B3D2BD7D74251431108E04051000883
:10146400006E41C501F0000E015604D040C500F0E5
:0614740041C501F0120069
:10147A0005013D6B3C5109081DE20A0E046E3CC58C
:10148A0000F071EC05F000C03DF500C03DF53D37B8
:10149A003D913D373D913D373D913D373D910A0E96
:1014AA00046E3CC500F071EC05F008C000F0005075
:0E14BA003D1302D03CC53DF53DC500F01200CB
:1014C800500E0301B46F000EB56F000EB66F000E1C
:1014D800B76F420EB86F010EB96F000EBA6F000EEB
:1014E800BB6F5C0EB06F020EB16F000EB26F000ED4
:1014F800B36F780EA86F030EA96F530EAA6F050E6F
:10150800AB6FB20EAC6F020EAD6F530EAE6F050E21
:10151800AF6F740E906F030E916F000E926F000EF6
:10152800936F959295908C928C90958295806D9EF4
:081538006D9C380E6C6E120070
:1015400028C504F029C505F026C502F027C503F01B
:101550002AC500F02BC501F0010E05012A5F000E1F
:101560002B5B005001100FE004C0E9FF05C0EAFF4B
:1015700002C0E1FF03C0E2FFEECFE6FF024A032A0A
:10158000044A052AE5D726C500F027C501F0120058
:101590003E0E05014A6F94EC03F00050200A01E171
:1015A0004BD0F2EC05F0020E05014A6F94EC03F00B
:1015B000BF0E001405014B6F020E4A6FADEC03F035
:1015C00005014A6B4B6BADEC03F0010E05014A6F50
:1015D000050E4B6FADEC03F0020E05014A6F200EB5
:1015E0004B6FADEC03F0030E05014A6F4B6BADEC96
:1015F00003F0040E05014A6F240E4B6FADEC03F0AF
:10160000050E05014A6F120E4B6FADEC03F0060E8E
:1016100005014A6F170E4B6FADEC03F0070E050185
:101620004A6F100E4B6FADEC03F03E0E05014A6F92
:0A163000200E4B6FADEC03F012002A
:10163A0005012A6B050E2A5D0AE22A512825E16E68
:10164A00000E2921E26E200EE66E2A2BF3D72A51CC
:10165A002825E16E000E2921E26EE66A2A072A5140
:10166A0028252B6F000E29212C6F0A0E046E000EFE
:10167A00056E26C500F027C501F0D7EC05F008C0B5
:10168A0000F009C001F0300E00262BC5E1FF2CC581
:10169A00E2FF00C0E6FF0A0E046E000E056E26C5C4
:1016AA0000F027C501F0D7EC05F000C026F501C00F
:1016BA0027F5000E011802E1000E001801E102D020
:0616CA002A07CDD7120033
:1016D000020E0B6E040E0C6EBA0E0D6E0D2EFED7A2
:0C16E0000C2EFCD70B2EFAD700001200D5
:1016EC0028C501F0010E006E015004E00036009098
:1016FC00FF0FFBD700C02AF5001E26C5E9FF27C542
:10170C00EAFF0050EF16120EE9260050EF1637DDF7
:10171C0005012A51EF12120EE95E5FDD2A51EF141A
:10172C00296F2951000A000ED8A4010E296F27DD5C
:06173C0029C500F01200B7
:10174200280E03017A6F000E7B6F5F0E7C6F050E11
:101752007D6FD20E886F010E896F000E8A6F000EA8
:101762008B6F820E8C6F000E8D6F000E8E6F000ECF
:101772008F6F9E0E846F000E856F000E866F000EB7
:10178200876FAC8A900EAB6E948E949C9EAA03D007
:08179200AECF00F0FBD71200FE
:10179A000900F5CFE6FF0006FBE10106F9E11200B8
:1017AA00826A0F013A6BFF0E946E948E949C82802B
:1017BA0094908B803F0E806E386B1E0E926E9286CE
:1017CA0092988998546BFF0E816E830E936E396BD3
:1017DA00836A3B6BFF0E956E95909482959C948ECE
:0417EA00606A12001F
:1017EE0026C500F00032009E0032009E0032009EA0
:1017FE000032009E330E0024F66E4D0EF76E000E74
:10180E00F722000EF86E000EF8220900F5CF00F058
:10181E0027C5E1FF28C5E2FF00C0E6FF010E050166
:10182E002725E16E000E2821E26E0F0E2615006EA2
:10183E00330E0024F66E4D0EF76E000EF722000EDC
:10184E00F86E000EF8220900F5CF00F000C0E6FF9A
:10185E00020E2725E16E000E2821E26EE66A1200C6
:10186E0028C5F6FF29C5F7FF2AC5F8FF0900F5CFF1
:10187E0000F0005218E028C5F6FF29C5F7FF2AC56B
:10188E00F8FF0900F5CF00F026C5E1FF27C5E2FFFE
:10189E0000C0E6FF0501264B272B010E2827000E60
:1018AE0029232A23DDD726C5E1FF27C5E2FFE66AF5
:0218BE00120016
:1018C00028C501F0010E006E015004E000360090C2
:1018D000FF0FFBD700C02CF5001C05012B6F2A6BF6
:1018E00026C5E9FF27C5EAFF296B2951070822E32E
:1018F0002B51EF16120EE9262B51EF16D4EC05F002
:101900002C51EF12D4EC05F0120EE95E2C51EF14BD
:10191000006E0CE029C501F0010E006E015004E0DC
:1019200000360090FF0FFBD700502A1357DC56DC1F
:0A193000292BDBD72AC500F01200B6
:0C193A00A60E0D6E0D2EFED70000120050
:1019460028C501F0010E006E015004E0003600903B
:10195600FF0FFBD700C02CF5001E00C02BF526C5D7
:10196600E9FF27C5EAFF0050EF16120EE92605012A
:101976002A6B2A51070815E32AC500F029C501F08C
:10198600005004E00132019EFF0FFBD72B51EF16EA
:1019960001A002D02C51EF1223DC2C51EF122A2B7E
:0C19A600E8D7120EE95E17DC16DC120018
:1019B2000A0E046E2AC500F071EC05F0300E002408
:1019C2000301CB6F0A0E046E2AC500F071EC05F01C
:1019D20008C000F0300E0024CC6F2F0ECD6F0A0E1F
:1019E200046EC8C300F071EC05F0300E0024CE6F17
:1019F2000A0E046EC8C300F071EC05F008C000F0D6
:101A0200300E0024CF6F2F0ED06F320ED16F300EFA
:101A1200D26F0A0E046E2CC500F071EC05F0300E88
:101A22000024D36F0A0E046E2CC500F071EC05F091
:101A320008C000F0300E0024D46FD56B0A0E046E7D
:101A420028C500F071EC05F0300E0024BE6F0A0EBE
:101A5200046E28C500F071EC05F008C000F0300EED
:101A62000024BF6F3A0EC06F0A0E046E27C500F045
:101A720071EC05F0300E0024C16F0A0E046E27C50A
:101A820000F071EC05F008C000F0300E0024C26FC7
:101A92003A0EC36F0A0E046E26C500F071EC05F013
:101AA200300E0024C46F0A0E046E26C500F071ECDD
:101AB20005F008C000F0300E0024C56FC66B12009E
:101AC200060E05012625E96E000E2721EA6EC00EDC
:101AD200EE24286F120EEE20296F000E2A6F2B6F54
:101AE20028C500F029C501F02AC502F02BC503F074
:101AF2000C0E046E000E056E066E076EFAEC08F010
:101B020000C028F501C029F502C02AF503C02BF553
:101B1200050E2625E96E000E2721EA6E030EEE5C05
:101B2200046E056A000E055A04500024386F0550F1
:101B32000120396F000E05BEFF0E02203A6F000E23
:101B420005BEFF0E03203B6F38C528F539C529F5C0
:101B52003AC52AF53BC52BF50C0E046E000E056E38
:101B6200066E076E38C500F039C501F03AC502F0BD
:101B72003BC503F023EC09F008C000F009C001F0F6
:101B82000AC002F00BC003F000C004F001C005F06F
:101B920002C006F003C007F004360490053606368C
:101BA2000736070E04240501346F000E0520356F39
:101BB200000E0620366F000E0720376F6D0E006E86
:101BC200010E016E000E026E036E38C504F039C5B7
:101BD20005F03AC506F03BC507F0FAEC08F03451BF
:101BE20000263551012236510222375103220C0EB2
:101BF200046E000E056E066E076E23EC09F000C03F
:101C020034F501C035F502C036F503C037F534C5E9
:101C12002CF535C52DF536C52EF537C52FF5030E36
:101C220005012625E96E000E2721EA6E300E046EAC
:101C3200000E056E066E076E38C500F039C501F05C
:101C42003AC502F03BC503F023EC09F0EE50002642
:101C5200000E012202220322530E005E7D0E015A63
:101C6200000E025A035A005005013425046E015039
:101C72003521056E02503621066E03503721076E5C
:101C820004C02CF505C02DF506C02EF507C02FF5B2
:101C9200800E000A006E800E0718005C08E10650F4
:101CA200230805E10550150802E1045023084FE21C
:101CB200C00E046E120E056E000E066E076E28C56B
:101CC20000F029C501F02AC502F02BC503F023EC70
:101CD20009F000C034F501C035F502C036F503C085
:101CE20037F5B00E046E040E056E000E066E076E1A
:101CF20028C500F029C501F02AC502F02BC503F062
:101D020023EC09F034C504F035C505F036C506F0FC
:101D120037C507F00050045E0150055A0250065ABA
:101D22000350075A260E0424006E000E0520016E91
:101D3200000E0620026E000E0720036E0050050101
:101D42002C2701502D2302502E2303502F23040E43
:101D52002625346F000E2721356F070E046E000E04
:101D6200056E066E076E2CC500F02DC501F02EC55E
:101D720002F02FC503F023EC09F008C000F009C0FF
:101D820001F00AC002F00BC003F034C5E1FF35C513
:101D9200E2FF00C0E6FF020E05012625E96E000EF5
:101DA2002721EA6EEECF30F5000E316F326F336FBE
:101DB200000E316F326F336F30C500F031C501F064
:101DC20032C502F033C503F0100E046E0E0E056E1E
:101DD200000E066E000E076EFAEC08F000C034F535
:101DE20001C035F502C036F503C037F534C530F50C
:101DF20035C531F536C532F537C533F5010E262521
:101E0200E96E000E2721EA6EEECF00F0000E016EA1
:101E1200026E036E3C0E046E000E056E000E066E20
:101E2200000E076EFAEC08F000503425046E0150E3
:101E32003521056E02503621066E03503721076E9A
:101E420004C030F505C031F506C032F507C033F5E0
:101E520026C5E9FF27C5EAFFEECF00F000500424B3
:101E6200346F000E0520356F000E0620366F000E0F
:101E72000720376F34C530F535C531F536C532F533
:101E820037C533F52CC500F02DC501F02EC502F083
:101E92002FC503F04950005E4A50015A4B50025A76
:101EA2004C50035A800E046E510E056E010E066EE2
:101EB200000E076EFAEC08F034510026355101226B
:0A1EC20036510222375103221200AC
:101ECC00A1EC00F0D00E0501536F59EC01F00501A7
:101EDC00536B59EC01F02EEC01F0D10E0501536F50
:101EEC0059EC01F0010E0501536FBCEC01F026C555
:101EFC00E1FF27C5E2FF00C0E6FF010E0501536FAD
:101F0C00BCEC01F028C5E1FF29C5E2FF00C0E6FFEB
:101F1C00010E0501536FBCEC01F02AC5E1FF2BC586
:101F2C00E2FF00C0E6FF010E0501536FBCEC01F0AF
:101F3C002CC5E1FF2DC5E2FF00C0E6FF010E050137
:101F4C00536FBCEC01F02EC5E1FF2FC5E2FF00C0C2
:101F5C00E6FF010E0501536FBCEC01F030C5E1FF4B
:101F6C0031C5E2FF00C0E6FF0501536BBCEC01F08C
:101F7C0032C5E1FF33C5E2FF00C0E6FFBAEC01F069
:021F8C00120041
:101F8E0026C504F027C505F004C002F005C003F015
:101F9E00044A052A28C500F029C501F00501284B81
:101FAE00292B00C0E9FF01C0EAFF02C0E1FF03C018
:101FBE00E2FFEECFE6FF02C0E9FF03C0EAFFEE52FA
:0E1FCE0001E0E2D726C500F027C501F01200A1
:101FDC0026C5E9FF27C5EAFFEECF03F0700E031408
:101FEC00026E02C000F00032009E0032009E0032F1
:101FFC00009E0032009E0A0E0002F3CF01F00F0E7D
:10200C000314006E26C5E1FF27C5E2FF0050012432
:10201C00E66E28C5E9FF29C5EAFFEECF03F0F00E06
:10202C000314026E02C000F00032009E0032009ECB
:10203C000032009E0032009E0A0E0002F3CF01F027
:10204C000F0E0314006E28C5E1FF29C5E2FF0050F6
:10205C000124E66E2AC5E9FF2BC5EAFFEECF03F09B
:10206C00300E0314026E02C000F00032009E0032EB
:10207C00009E0032009E0032009E0A0E0002F3CF3A
:10208C0001F00F0E0314006E2AC5E1FF2BC5E2FF11
:10209C0000500124E66E2CC5E9FF2DC5EAFF2CC5C6
:1020AC00E1FF2DC5E2FF070EEE162EC5E9FF2FC589
:1020BC00EAFFEECF03F0F00E0314026E02C000F044
:1020CC000032009E0032009E0032009E0032009EC4
:1020DC000A0E0002F3CF01F00F0E0314006E2EC592
:1020EC00E1FF2FC5E2FF00500124E66E30C5E9FF89
:1020FC0031C5EAFFEECF03F0100E0314026E02C0DE
:10210C0000F00032009E0032009E0032009E003231
:10211C00009E0A0E0002F3CF01F00F0E0314006EA6
:10212C0030C5E1FF31C5E2FF00500124E66E32C537
:10213C00E9FF33C5EAFFEECF03F0F00E0314026E95
:10214C0002C000F00032009E0032009E0032009E61
:10215C000032009E0A0E0002F3CF01F00F0E0314A2
:10216C00006E32C5E1FF33C5E2FF00500124E66E7C
:02217C0012004F
:0E217E009488949A94968298829A829612007F
:10218C000F0E05013C6F3D6B3E6B3F6B406B416B23
:10219C00426B436B446B78EC08F0090E05013C6F05
:1021AC003D6B3E6B3F6B406B416B426B436B446BC7
:1021BC0078EC08F00A0E05013C6F010E3D6F010E24
:1021CC003E6F010E3F6F010E406F010E416F010E0D
:1021DC00426F010E436F010E446F78EC08F00B0E4A
:1021EC0005013C6F070E3D6F070E3E6F070E3F6FEC
:1021FC00070E406F070E416F070E426F070E436FBD
:10220C00070E446F78EC08F00C0E05013C6F010EC4
:10221C003D6F010E3E6F010E3F6F010E406F010EC0
:10222C00416F010E426F010E436F010E446F78EC4B
:10223C0008F01A0E0C6EF80E0D6E0D2EFED70C2E2D
:10224C00FCD70000B5EC05F0020E0B6E040E0C6E04
:10225C00BA0E0D6E0D2EFED70C2EFCD70B2EFAD708
:04226C00000012005C
:10227000210ECD6ECD823C0ECF6EB00ECE6E9E90F6
:102280009F900401C66BC76B0301BC6BBD6BCD9007
:042290009D9012000B
:1022940026C5F6FF27C5F7FF28C5F8FF0900F5CFC7
:1022A40001F00150000817E28B9026C5F6FF27C500
:1022B400F7FF28C5F8FF0900F5CF3CF529C53DF522
:1022C4002AC53EF50DEC06F0010E2627000E272345
:0822D40028238B80DDD71200E6
:1022DC003C0ECF6EB00ECE6E0401C66BC76B030105
:0C22EC00BC6BBD6BCD809D809E901200ED
:1022F800000E0501271902E1000E261937E026C550
:10230800E9FF27C5EAFFEE5231E028C53CF529C5AB
:102318003DF523EC08F000C040F526C53CF527C57F
:102328003DF528C53EF529C53FF5A7EC07F0000E99
:10233800011802E1000E001805E126C500F027C5C6
:1023480001F016D0010E050126253C6F000E27214D
:102358003D6F28C5E9FF29C5EAFFEECF3EF5D0EC71
:1023680008F000C026F501C027F5C2D7006A016A47
:02237800120051
:10237A000501296B030E295D0AE229512725E16E21
:10238A00000E2821E26E200EE66E292BF3D7295182
:10239A002725E16E000E2821E26EE66A29072951F7
:1023AA0027252A6F000E28212B6F0A0E046E26C5D8
:1023BA0000F071EC05F008C000F0300E00262AC5C6
:1023CA00E1FF2BC5E2FF00C0E6FF0A0E046E26C538
:1023DA0000F071EC05F000C026F50050000A01E19A
:0823EA0002D02907DCD7120024
:1023F20027C500F00032009E0032009E0032009E8F
:102402000032009E330E0024F66E4D0EF76E000E63
:10241200F722000EF86E000EF8220900F5CF00F048
:1024220028C5E1FF29C5E2FF00C0E6FF010E050154
:102432002825E16E000E2921E26E0F0E2715006E8F
:10244200330E0024F66E4D0EF76E000EF722000ECC
:10245200F86E000EF8220900F5CF00F000C0E6FF8A
:10246200020E2825E16E000E2921E26E26C500F03B
:102472000032009E0032009E0032009E0032009E1A
:10248200330E0024F66E4D0EF76E000EF722000E8C
:10249200F86E000EF8220900F5CF00F000C0E6FF4A
:1024A200030E2825E16E000E2921E26E0F0E26157D
:1024B200006E330E0024F66E4D0EF76E000EF722FC
:1024C200000EF86E000EF8220900F5CF00F000C0F1
:1024D200E6FF040E2825E16E000E2921E26EE66A6F
:0224E2001200E6
:1024E4000501286B296BAAEC05F0DD0E05013C6F94
:1024F400030E3D6F23EC08F000C026F501C027F55C
:102504000301DD51550AD8A4C7D0F051230AD8A439
:10251400C3D0800E05012719006E800E005C02E115
:10252400140E265DD8A0B8D0580E3C6F4C0E3D6FEB
:10253400000E3E6F8CEC05F0DD0E05013C6F030EC2
:102544003D6F8CEC07F0020E2A6F000E2B6F800E8D
:102554002B19006E800E2719005C02E126512A5DBA
:102564002FE2DD0E2A25E96E030E2B21EA6EEECF53
:1025740001F001503B0A21E1DD0E2A25E16E030E34
:102584002B21E26EE66A5D0E28252C6F040E2921AC
:102594002D6FDD0E2A253C6F030E2B213D6F020E9D
:1025A4003C5F000E3D5BD2EC09F02CC5E1FF2DC56C
:1025B400E2FF00C0E6FF284B292B2A4B2B2BC7D761
:1025C4000301F06B5D0E05012825E16E040E29213F
:1025D400E26E300E0301EE5D006E0A0E0002F3CFD0
:1025E40000F0EF510026300E005E00C0E6FF5DC42F
:1025F4003CF53DEC0AF000C0C8F45EC43CF53DEC8B
:102604000AF000C0C8F35FC43CF53DEC0AF000C01A
:10261400C9F460C43CF53DEC0AF000C0C5F461C4E3
:102624003CF53DEC0AF000C0C9F362C43CF53DEC56
:102634000AF000C0DCF30301DB6BDB6BAAEC05F0F2
:1026440007EC07F0DBC33CF5000E05013D6FDCC36E
:102654003EF5000E3F6FC9C340F5000E416FC5C47F
:1026640042F5000E436FC8C444F5000E456FC8C35D
:1026740046F5000E476FC9C448F5000E496FD8EC03
:1026840007F0110E05013C6F4D0E3D6F000E3E6FBD
:0A2694008CEC05F0F2EC05F01200EA
:10269E0005012A6B2B6B28512A253C6F29512B21C2
:1026AE003D6FCAEC05F000C02CF5000E2D6F000E2C
:1026BE002D1902E1000E2C1901E124D0800E006EBE
:1026CE00800E2B19005C02E12A513F0801E21AD05C
:1026DE002A512625E16E2B512721E26E2CC5E6FFED
:1026EE00030E0C6E970E0D6E0D2EFED70C2EFCD714
:1026FE00000000002A4B2B2B000E2D1902E1000EBC
:10270E002C19C9E12A512625006E2B512721016E65
:10271E00010E005CE16E000E0158E26EE66A1200D8
:10272E009F8A0001E66BE76B800EE719006E800E44
:10273E00000A005C02E17F0EE65D12E2DD0EE62588
:10274E00E16E030EE721E26EE66A010EE625006EEB
:10275E00000EE721016E00C0E6F001C0E7F0E4D7FD
:10276E00E86BE96BE66BE76BE56BE16BE26B9D8A01
:06277E00E36BE46B1200A6
:1027840026C504F027C505F004C0E9FF05C0EAFF2B
:10279400EE5203E0044A052AF7D704C002F005C04C
:1027A40003F0044A052A28C500F029C501F00501F3
:1027B400284B292B00C0E9FF01C0EAFF02C0E1FF5A
:1027C40003C0E2FFEECFE6FF02C0E9FF03C0EAFF69
:1027D400EE5201E0E2D726C500F027C501F0120051
:1027E40005012E6B2F6B26C530F527C531F528C59D
:1027F40032F529C533F5800E2919006E800E005C70
:1028040008E1000E285D05E1000E275D02E1000EDF
:10281400265D10E2010E2E6F000E2F6F306B316BB0
:10282400326B336B2651305F2751315B2851325B59
:102834002951335B30C53CF531C53DF532C53EF514
:1028440033C53FF52AC540F52BC541F51BEC07F010
:102854000B0E2C6F000E2D6F000E006E2D51005CC0
:1028640002E12C51000819E22C512A25E16E2D5168
:102874002B21E26E010E2C5D006E000E2D59016EAF
:1028840000502A25E96E01502B21EA6EEECFE6FFB7
:10289400010E2C5F000E2D5BDFD72AC5E1FF2BC58F
:1028A400E2FF200EE66E2E512F111AE02C6B2D6BD9
:1028B4002C512A25E96E2D512B21EA6EEE50200A67
:1028C40003E12C4B2D2BF4D7010E2C5F000E2D5B56
:1028D4002C512A25E16E2D512B21E26E2D0EE66E30
:0228E4001200E0
:1028E600050127AF09D02D0E0401756F0501261FBE
:1028F600271F264B272B03D0200E0401756F26C5F4
:1029060000F027C501F001320032019E013200328B
:10291600019E01320032019E01320032019E00C04A
:1029260028F50A0E046E71EC05F00A0E046E71ECC1
:1029360005F008C000F0300E0024016E01C076F4E8
:102946000150300A03E10401200E766F04010A0EDD
:10295600046E28C500F071EC05F008C000F0300EDA
:102966000024776F26C529F527C52AF50F0E050120
:102976002615006E27C501F0000E011600C029F5C8
:1029860001C02AF5710E046E020E056E1DEC04F0F0
:1029960000C02BF501C02CF52BC529F52CC52AF551
:1029A6002E0E0401786FE80E046E030E056E2BC51D
:1029B60000F02CC501F0D7EC05F0300E0024796F3D
:1029C600640E046E000E056E2BC500F02CC501F0DA
:1029D600D7EC05F00A0E046E000E056ED7EC05F076
:1029E60008C000F009C001F0300E00247A6F0A0E0C
:1029F600046E000E056E2BC500F02CC501F0D7EC59
:102A060005F00A0E046E000E056ED7EC05F008C040
:102A160000F009C001F0300E00247B6F7A6B7C6BEE
:102A26007D6B760E05013C6F040E3D6F40EC08F0A1
:102A360028C500F0000E016EE80E046E030E056E4A
:102A46001DEC04F0295100245A6E2A5101205B6EB8
:082A5600000E5C6E5D6E1200C3
:102A5E0026C53CF527C53DF523EC08F026C5E9FF54
:102A6E0027C5EAFFEE50000811E28B9026C5E9FF5C
:102A7E0027C5EAFFEECF3CF528C53DF529C53EF545
:102A8E000DEC06F0264B272B8B80E8D78B8012009F
:102A9E0000C01AF001C019F0E1CF1BF0E2CF1CF01C
:102AAE009DAA65D09EAA63D0AECFE5F0ABA20FD0A3
:102ABE00AB98AECFE5F0AB88010E03017E25006E1C
:102ACE00000E7F21016E00C07EF301C07FF3ABA428
:102ADE000FD00301AB9EAB8E010E7E25006E000E55
:102AEE007F21016E00C07EF301C07FF3AECFE5F013
:102AFE000001E5510D0A07E0E951000802E1E85135
:102B0E007E0801E314D0010EE16F000EE26F9D9A74
:102B1E00DD0EE825E16E030EE921E26EE66AE8C0FD
:102B2E00E6F0E9C0E7F0E86BE96BE56B20D0E95120
:102B3E00000802E1E8517E0804E2020EE16F000E89
:102B4E00E26FDD0EE825E16E030EE921E26EE5C0CF
:102B5E00E6FFE8C0E6F0E9C0E7F0010EE825006EFA
:102B6E00000EE921016E00C0E8F001C0E9F0F2AA02
:102B7E000AD0F2A408D0010E03018027000E812393
:102B8E0082238323F2941AC000F019C001F01BC0F7
:082B9E00E1FF1CC0E2FF110081
:102BA60000C018F0156ED8CF16F0E0CF17F09DA034
:102BB6001ED09EA01CD00401C64BC72B03016F512B
:102BC6000401C75D04E103016E510401C65D0AE319
:102BD6009D90C66BC76B010E0301BC6F000EBD6FE7
:102BE600CD909D900B0ECF6EDB0ECE6E9E90175045
:102BF600E06E1650D86E153A153818C000F0100061
:102C0600FCEC26F09B6A600ED36E9B9CD26A640E27
:102C1600476E000E486ED5EC0BF08B80020E0B6EE5
:102C2600040E0C6EBA0E0D6E0D2EFED70C2EFCD7B2
:102C36000B2EFAD70000080E03016E6F000E6F6FA1
:102C46008998B886B06A670EAF6EAC84A1EC0BF0BB
:102C5600020E0B6E040E0C6EBA0E0D6E0D2EFED706
:102C66000C2EFCD70B2EFAD700000C0E05015F6F59
:102C760014EC00F0060E0B6E130E0C6EAD0E0D6E00
:102C86000D2EFED70C2EFCD70B2EFAD70000000017
:102C9600EA0E03016C6F020E6D6F7D0E6A6F000EF9
:102CA6006B6FAAEC05F0D90E05013C6F4C0E3D6F1B
:102CB600000E3E6F8CEC05F00001696B6A6B000E2E
:102CC6006A5D02E1080E695D1CE2030E006E000EED
:102CD600016E69C004F06AC005F01DEC04F01D0E1B
:102CE6000024E96E000E0120EA6EEECF3CF5EECF31
:102CF6003DF5EECF3EF58CEC05F00001694B6A2BF5
:102D0600DED70B0E0B6E260E0C6E5D0E0D6E0D2EA7
:102D1600FED70C2EFCD70B2EFAD700000000AAEC2B
:102D260005F0B20E05013C6F4C0E3D6F000E3E6F76
:102D36008CEC05F068EC0BF00001676B686B800E9D
:102D46000501266F0F0E276F286B76EC0BF09DECB6
:102D56000CF0800E266F0F0E276F286B330E296F2F
:102D6600A3EC0CF09DEC0CF0800E266F0F0E276F77
:102D7600286B60EC0CF000C0E5F09DEC0CF0430E07
:102D86003C6F4D0E3D6F000E3E6F8CEC05F004015E
:102D9600756BE5C026F5750E0501276F040E286FC5
:102DA600F7EC0BF0750E3C6F040E3D6F8CEC07F0E4
:102DB600DC0E3C6F4D0E3D6F000E3E6F8CEC05F049
:102DC6000001696B6A6B000E6A5D02E1060E695DC1
:102DD6002AE2800E0501266F0F0E276F286B60EC26
:102DE6000CF000C0E5F09DEC0CF05E0E00016925CC
:102DF600E16E000E6A21E26EE5C0E6FF0401756B26
:102E0600E5C026F5750E0501276F040E286FF7EC51
:102E16000BF0750E3C6F040E3D6F8CEC07F0000155
:102E2600694B6A2BD0D7C60E05013C6F4D0E3D6F20
:102E3600000E3E6F8CEC05F0800E0501266F0F0E1E
:102E4600276F286B60EC0CF000C0E5F00401756B91
:102E5600E5C026F5750E0501276F040E286FF7EC01
:102E66000BF0750E3C6F040E3D6F8CEC07F0AAEC70
:102E760005F0400E0001656F1F0E666F6CC326F5E8
:102E86006DC327F5C20E0501286F4B0E296F000E84
:102E96002A6F37EC0CF065C026F566C027F5750E6F
:102EA6000501286F040E296F1DEC0BF0170E0301A8
:102EB6006C250501266F000E03016D210501276FA4
:102EC600750E286F040E296F050E2A6F000E2B6FE4
:102ED600A0EC0AF06CC33CF56DC33DF58CEC07F035
:102EE6000301CA6B050E6E6E64EC0AF0000E050156
:102EF6003C6F490E3D6F000E3E6F8CEC05F0C8EC42
:102F06000AF0F2EC05F0060E0B6E130E0C6EAD0E0B
:102F16000D6E0D2EFED70C2EFCD70B2EFAD7000009
:102F26000000DBC326F5DCC327F5C9C328F5C5C4F5
:102F360029F5C8C42AF5C8C32BF5C9C42CF5D9ECA4
:102F46000CF0610E05013C6F4D0E3D6F000E3E6F9D
:102F56008CEC05F0CB0E05013C6F030E3D6F8CEC3F
:102F660007F0BE0E3C6F4D0E3D6F000E3E6F8CECB3
:102F760005F0BE0E05013C6F030E3D6F8CEC07F0AD
:102F8600AAEC05F0060E0B6E130E0C6EAD0E0D6E52
:102F96000D2EFED70C2EFCD70B2EFAD70000000004
:102FA6003B0E00016B6F370E6C6F120E6D6F150EB8
:102FB6006E6F0C0E706FE20E716F070E726F756B8F
:102FC600766B776B010E786F010E7A6FE30E7B6F6F
:102FD600070E7C6F9C0E05013C6F4B0E3D6F000E7D
:102FE6003E6F8CEC05F06B0E0501266F000E276F09
:102FF60061EC0DF000C043F001C044F002C045F0A2
:1030060003C046F000C03CF501C03DF502C03EF5E8
:1030160003C03FF5750E406F040E416F1BEC07F0C1
:10302600750E3C6F040E3D6F8CEC07F0AAEC05F0B4
:10303600760E05013C6F4B0E3D6F000E3E6F8CEC1D
:1030460005F0750E0501266F000E276F61EC0DF079
:1030560000C03FF001C040F002C041F003C042F0A2
:1030660000C03CF501C03DF502C03EF503C03FF58A
:10307600750E406F040E416F1BEC07F0750E3C6F2A
:10308600040E3D6F8CEC07F0AAEC05F06F0E0501FF
:103096003C6F4D0E3D6F000E3E6F8CEC05F0750ECD
:1030A6000501266F000E276F61EC0DF000C022F5BA
:1030B60001C023F502C024F503C025F56B0E266F6B
:1030C600000E276F61EC0DF022C504F023C505F054
:1030D60024C506F025C507F00050045E0150055AC8
:1030E6000250065A0350075A04C03BF005C03CF094
:1030F60006C03DF007C03EF004C03CF505C03DF5F6
:1031060006C03EF507C03FF5750E406F040E416FD1
:103116001BEC07F0750E3C6F040E3D6F8CEC07F050
:10312600AAEC05F0580E05013C6F4A0E3D6F000EE5
:103136003E6F8CEC05F0BFEC10F08B80C6EC10F007
:103146006F0E3C6F4C0E3D6F000E3E6F8CEC05F023
:10315600B5EC05F0020E0B6E040E0C6EBA0E0D6E7B
:103166000D2EFED70C2EFCD70B2EFAD70000B5EC91
:1031760005F09F90F28CD08EF28CF28ED08EF28E6D
:103186009F80780E3C6F490E3D6F000E3E6F8CECB3
:1031960005F0140E03016E6F000E6F6F38EC11F020
:1031A6006EEC11F0240EAD6EAAEC05F0000E0301D4
:1031B600BD1902E1000EBC1901E1F8D7230EAD6E70
:1031C600AAEC05F00001736B746B8A0E05013C6F67
:1031D6004A0E3D6F000E3E6F8CEC05F0C6EC10F00B
:1031E600B5EC05F00A0E4A6F010E4B6F010E4C6FDF
:1031F600010E4D6F010E4E6F010E4F6F010E506F97
:10320600010E516F010E526FE0EC03F0B5EC05F0C4
:103216007C0E266F4D0E276F000E286F070E296F46
:10322600000E2A6F4AEC11F00B0E0B6E260E0C6E7A
:103236005D0E0D6E0D2EFED70C2EFCD70B2EFAD77B
:10324600000000000A0E03016E6F000E6F6FEA0E9B
:103256006C6F020E6D6F708B596A280E476E000EEA
:10326600486EF29EC6EC10F0B5EC05F0CE0E266F59
:103276004D0E276F000E286F47C029F548C02AF566
:103286004AEC11F07D0E03016A6F000E6B6FEA0EB9
:103296006C6F020E6D6FDB0E0501266F030E276F36
:1032A600DC0E286F030E296FC90E2A6F030E2B6FD3
:1032B600C50E2C6F040E2D6FC80E2E6F040E2F6FC9
:1032C600C80E306F030E316FC90E326F040E336FA6
:1032D60066EC0FF0DB0E0501266F030E276FDC0E82
:1032E600286F030E296FC90E2A6F030E2B6FC50EAA
:1032F6002C6F040E2D6FC80E2E6F040E2F6FC80E86
:10330600306F030E316FC90E326F040E336FEEEC61
:103316000FF0DBC326F5DCC327F5C9C328F5C5C402
:1033260029F5C8C42AF5C8C32BF5C9C42CF5D9ECB0
:103336000CF03B0E0001756F3B0E766F170E776F24
:103346001F0E786F0C0E7A6FE20E7B6F070E7C6F86
:10335600DBC36BF0DCC36CF0C9C36DF0C8C46EF0A0
:10336600C8C370F0D00E006E070E016E0401C9517D
:103376000026D8B0012A00C071F001C072F0EA0E32
:1033860003016C6F020E6D6F6CC326F56DC327F5D6
:10339600CB0E0501286F030E296FC7EC0FF06CC327
:1033A6003CF56DC33DF523EC08F000C073F001C099
:1033B60074F0005003016C250501266F01500301CE
:1033C6006D210501276F200E0401CA6FCB6BCA0E53
:1033D6000501286F040E296FC2EC13F06CC33CF58F
:1033E6006DC33DF523EC08F000C073F001C074F026
:1033F600005003016C250501266F015003016D2164
:103406000501276FBE0E286F030E296FC2EC13F05D
:103416006B0E266F000E276F61EC0DF000C043F0B7
:1034260001C044F002C045F003C046F0750E266F99
:10343600000E276F61EC0DF000C03FF001C040F0B8
:1034460002C041F003C042F0750E266F000E276FD2
:1034560061EC0DF000C022F501C023F502C024F591
:1034660003C025F56B0E266F000E276F61EC0DF07D
:1034760022C53BF023C53CF024C53DF025C53EF0F2
:1034860000503B5E01503C5A02503D5A03503E5A92
:1034960097EC13F0F28E80B698D0230E05013C6FA0
:1034A6004D0E3D6F000E3E6F8CEC05F043C03CF5B3
:1034B60044C03DF545C03EF546C03FF5750E0501D5
:1034C600406F040E416F1BEC07F0750E3C6F040E47
:1034D6003D6F8CEC07F0AAEC05F0E60E05013C6F9B
:1034E6004B0E3D6F000E3E6F8CEC05F03FC026F58F
:1034F60040C027F541C028F542C029F5750E0501E3
:103506002A6F040E2B6FF2EC13F0750E3C6F040E4F
:103516003D6F8CEC07F0AAEC05F0520E05013C6FEE
:103526004D0E3D6F000E3E6F8CEC05F03BC026F550
:103536003CC027F53DC028F53EC029F5960E05018D
:103546002A6F030E2B6FF2EC13F0960E3C6F030EF0
:103556003D6F40EC08F0960E3C6F030E3D6F8CEC11
:1035660007F0950E3C6F4D0E3D6F000E3E6F8CECD6
:1035760005F0100E046E0E0E056E000E066E076E3A
:103586003BC000F03CC001F03DC002F03EC003F07D
:1035960023EC09F000C073F001C074F000C026F5FA
:1035A60001C027F5750E0501286F040E296F1DEC65
:1035B6000BF0750E3C6F040E3D6F8CEC07F0480E59
:1035C6005F6F14EC00F0AAEC05F0800E3E18006E5A
:1035D600800E005C08E1000E3D5C05E1000E3C5CDF
:1035E60002E1040E3B5C40E27F0E006E800E3E1848
:1035F600005C08E13D50FF0805E13C50FF0802E190
:103606003B50880831E20F0E03016E6F000E6F6F9C
:103616006AC326F56BC327F51C0E0501286F4B0EF2
:10362600296F000E2A6F37EC0CF06AC33CF56BC3AA
:103636003DF58CEC07F0AAEC05F06AC326F56BC3E2
:1036460027F547C028F548C029F52FEC15F0030EDD
:103656000B6E080E0C6E770E0D6E0D2EFED70C2E11
:10366600FCD70B2EFAD7C0D0800E006E800E3E1807
:10367600005C08E13D50000805E13C50000802E10D
:103686003B50040856E2800E3E18006E800E005C29
:1036960008E1000E3D5C05E1010E3C5C02E12C0EEA
:1036A6003B5C47E20F0E476E000E486E0A0E0301A2
:1036B6006E6F000E6F6F7D0E6A6F000E6B6F6AC3C2
:1036C60026F56BC327F5F40E0501286F4D0E296FFD
:1036D600000E2A6F37EC0CF06AC326F56BC327F58C
:1036E600960E0501286F030E296FC2EC13F06AC30C
:1036F60026F56BC327F5200E0401CC6F530ECD6F54
:10370600650ECE6F630ECF6F200ED06FD16BCC0ED1
:103716000501286F040E296FC2EC13F06AC326F563
:103726006BC327F547C028F548C029F52FEC15F0DF
:103736005BD01E0E476E000E486E0F0E03016E6FB5
:10374600000E6F6FEA0E6C6F020E6D6F6CC326F57E
:103756006DC327F5CB0E0501286F030E296FC7EC45
:103766000FF06CC33CF56DC33DF523EC08F000C0CB
:1037760073F001C074F0005003016C250501266F3B
:10378600015003016D210501276F200E0401D26F40
:10379600D36BD20E0501286F040E296FC2EC13F00D
:1037A6006CC33CF56DC33DF523EC08F000C073F027
:1037B60001C074F0005003016C250501266F01500D
:1037C60003016D210501276FBE0E286F030E296FB9
:1037D600C2EC13F06CC326F56DC327F547C028F578
:1037E60048C029F52FEC15F0B5EC05F0B50E266F9F
:1037F6004D0E276F000E286F47C029F548C02AF5E1
:103806004AEC11F0800E0501266F0F0E276F286B0C
:1038160076EC0BF0800E266F0F0E276F286BCC0E02
:10382600296FA3EC0CF0800E266F0F0E276F286B06
:10383600440E296FA3EC0CF09DEC0CF0800E266F65
:103846000F0E276F286B76EC0BF0800E266F0F0E8F
:10385600276F286BCC0E296FA3EC0CF0800E266F19
:103866000F0E276F286BBE0E296FA3EC0CF0800E8F
:10387600266F0F0E276F286B60EC0CF000C057F018
:10388600000E586E800E266F0F0E276F286B60ECA9
:103896000CF000C003F0026A57500224006E585024
:1038A6000320016E00C055F001C056F000C026F599
:1038B60001C027F573EC14F0750E3C6F040E3D6FD6
:1038C60040EC08F0750E3C6F040E3D6F23EC08F0DB
:1038D60000C073F001C074F0750E0024266F040E4C
:1038E6000120276FEF0E286F4D0E296F000E2A6FED
:1038F60037EC0CF0750E05013C6F040E3D6F8CEC39
:1039060007F0AAEC05F0750E05013C6F040E3D6F3D
:1039160023EC08F000C073F001C074F00001696B7D
:103926006A6B74516A5D02E17351695D14E2750E4A
:103936006925E96E040E6A21EA6EEE50B00A08E1C6
:10394600750E6925E16E040E6A21E26E7E0EE66E44
:10395600694B6A2BE6D7010E5914016E0150010A14
:1039660019E1B5EC05F0E30E266F4D0E276F000E3C
:10397600286F010E296F000E2A6F4AEC11F0750EA2
:103986000501266F040E276F47C028F548C029F5A4
:103996002FEC15F00501A00E3C6F4D0E3D6F000E8D
:1039A6003E6F8CEC05F059C026F5750E0501276FA4
:1039B600040E286FBDEC11F0750E3C6F040E3D6FC2
:1039C6008CEC07F0AAEC05F0592A0A0E03016E6F7B
:1039D600000E6F6F38EC11F06EEC11F00301000E63
:1039E600BD1902E1000EBC1908E1000E0001E21942
:1039F60002E1000EE11901E1F1D70001000EE21922
:103A060002E1010EE119D8A416EF21F0DD0E050141
:103A16003C6F030E3D6F8CEC07F0AAEC05F0DD0E53
:103A26000501266F030E276F4D0E0401D46F730E2A
:103A3600D56F670ED66F3D0ED76FD86BD40E0501C6
:103A4600286F040E296F7CEC11F000C0E3F001C072
:103A5600E4F0000E026E0150025C02E10050000824
:103A660053E2DD0E05013C6F030E3D6F23EC08F0BB
:103A7600800E026E800E0118025C02E100500608FC
:103A860043E2DD0E3C6F030E3D6F23EC08F000C0F1
:103A960073F001C074F0000E026E0150025C02E188
:103AA6000050060831E2000E0001745D02E17A0E54
:103AB600735D2AE2EA0EF66E470EF76E000EF86E9A
:103AC600D90EE16E040EE26E190E006E010E016E45
:103AD600CDEC0BF0D90E05013C6F040E3D6F8CEC5E
:103AE60007F0E10E3C6F030E3D6F8CEC07F0AAEC7D
:103AF60005F06CC326F56DC327F5E10E0501286FA9
:103B0600030E296FC7EC0FF00501DD0E266F030EBD
:103B1600276F540E0401F26F450EF36F4D0EF46FCE
:103B2600500EF56F5F0EF66F4F0EF76F4E0EF86F75
:103B3600F96BF20E0501286F040E296F7CEC11F06B
:103B460000C0E3F001C0E4F0000E026E0150025C1A
:103B560002E10050000815E20301708BDD0E05013D
:103B66003C6F030E3D6F23EC08F000C073F001C0FC
:103B760074F09C0E3C6F4C0E3D6F000E3E6F8CEC4D
:103B860005F0DD0E0501266F030E276F540E0401A6
:103B9600FA6F450EFB6F4D0EFC6F500EFD6F5F0EFC
:103BA600FE6F4F0EFF6F460E0501006F460E016F4A
:103BB600026BFA0E286F040E296F7CEC11F000C020
:103BC600E3F001C0E4F0000E026E0150025C02E177
:103BD600005000080BE20301709BED0E05013C6FDF
:103BE6004A0E3D6F000E3E6F8CEC05F0DD0E0501B2
:103BF600266F030E276F530E036F700E046F650E4C
:103C0600056F650E066F640E076F3D0E086F096B34
:103C1600030E286F050E296F7CEC11F000C0E3F04F
:103C260001C0E4F0000E026E0150025C02E1005099
:103C36000008D8B08AD0DD0E05013C6F030E3D6F3B
:103C460023EC08F000C073F001C074F0000E026EA1
:103C56000150025C02E100500608D8B076D003019C
:103C6600946B956B0001696B6A6B060E735D016E52
:103C7600000E7459026E02506A5D02E10150695DE0
:103C86001DE2E30E6925E96E030E6A21EA6EEECFA8
:103C960001F0300E015C0EE3E30E6925E96E030EBA
:103CA6006A21EA6EEECF01F00150390803E3030101
:103CB600944B952B0001694B6A2BD7D7060E735D83
:103CC600016E000E7459026E03019551021802E14D
:103CD600015094193AE1E30E05013C6F030E3D6F66
:103CE600D2EC09F000C0A6F301C0A7F3000E026EE5
:103CF6000150025C02E1005001080BE2000E0301D4
:103D0600A75D02E1FF0EA65D04E2A6C347F0A7C3C6
:103D160048F0C60E05013C6F4C0E3D6F000E3E6F1F
:103D26008CEC05F047C026F548C027F5750E050151
:103D3600286F040E296F1DEC0BF0750E3C6F040EF8
:103D46003D6F8CEC07F0AAEC05F0DD0E0501266F41
:103D5600030E276F450E0A6F650E0B6F700E0C6F04
:103D6600720E0D6F6F0E0E6F6D0E0F6F3D0E106F94
:103D7600116B0A0E286F050E296F7CEC11F000C03E
:103D8600E3F001C0E4F0000E026E0150025C02E1B5
:103D960000500008D8B0C1D0DD0E05013C6F030EFF
:103DA6003D6F23EC08F000C073F001C074F0000E04
:103DB600026E0150025C02E100500708D8B0ADD097
:103DC600000E0001745D02E10A0E735DD8B0A5D045
:103DD6000301946B956B0001696B6A6B070E735D4B
:103DE600016E000E7459026E02506A5D02E10150C6
:103DF600695D1DE2E40E6925E96E030E6A21EA6E2D
:103E0600EECF01F0300E015C0EE3E40E6925E96E9B
:103E1600030E6A21EA6EEECF01F00150390803E382
:103E26000301944B952B0001694B6A2BD7D7070EDC
:103E3600735D016E000E7459026E030195510218EE
:103E460002E10150941969E1E40E05013C6F030E8D
:103E56003D6FD2EC09F000C0A6F301C0A7F3D50E62
:103E66003C6F4D0E3D6F000E3E6F8CEC05F0A6C309
:103E760026F5A7C327F5750E0501286F040E296FD1
:103E86001DEC0BF0750E3C6F040E3D6F8CEC07F0CD
:103E9600090E5F6F14EC00F0000E0301A75D02E14E
:103EA600000EA65D3AE3000EA75D02E1100EA65DC8
:103EB60034E2060E006EA6C373F0A7C374F000507A
:103EC60006E00001733773917437FF0FF9D7860E3A
:103ED60005013C6F4C0E3D6F000E3E6F8CEC05F0FD
:103EE60073C026F574C027F5750E0501286F040EFC
:103EF600296FF9EC11F0750E3C6F040E3D6F8CECDA
:103F060007F0AAEC05F06CC326F56DC327F573C060
:103F160028F574C029F54FEC13F00301DD51550A5D
:103F2600D8A483D0F051230AD8A47FD04A0E050125
:103F36003C6F4B0E3D6F000E3E6F8CEC05F072EC45
:103F460012F0DB0E0501266F030E276FDC0E286FBD
:103F5600030E296FC90E2A6F030E2B6FC50E2C6F29
:103F6600040E2D6FC80E2E6F040E2F6FC80E306F05
:103F7600030E316FC90E326F040E336F66EC0FF00D
:103F8600DB0E0501266F030E276FDC0E286F030E6E
:103F9600296FC90E2A6F030E2B6FC50E2C6F040EE8
:103FA6002D6FC80E2E6F040E2F6FC80E306F030EC6
:103FB600316FC90E326F040E336FEEEC0FF0DBC3B8
:103FC60026F5DCC327F5C9C328F5C5C429F5C8C439
:103FD6002AF5C8C32BF5C9C42CF5D9EC0CF0FF0E95
:103FE60005013C6F4C0E3D6F000E3E6F8CEC05F0EC
:103FF600CB0E05013C6F030E3D6F8CEC07F0890E6E
:104006003C6F4D0E3D6F000E3E6F8CEC05F0BE0E04
:1040160005013C6F030E3D6F8CEC07F0AAEC05F032
:104026000301DD6B0001E36BE46BDD0E0501266F1A
:10403600030E276F440E126F650E136F6D0E146F0D
:104046006F0E156F166B120E286F050E296F7CEC1E
:1040560011F000C0E3F001C0E4F0000E026E015062
:10406600025C02E1005000086EE2EB0E05013C6FB7
:10407600490E3D6F000E3E6F8CEC05F00001696B3A
:104086006A6B000E6A5D02E10F0E695D5CE2060E68
:10409600026E69C000F06AC001F0025005E0003609
:1040A60000900136FF0FFAD700C073F001C074F01C
:1040B6006CC326F56DC327F500C028F501C029F5A8
:1040C6004FEC13F0AB0E3C6F4D0E3D6F000E3E6F86
:1040D6008CEC05F073C026F574C027F5750E050146
:1040E600286F040E296FF9EC11F0750E3C6F040E63
:1040F6003D6F8CEC07F0090E5F6F14EC00F06CC39B
:104106003CF56DC33DF58CEC07F0AAEC05F06CC3ED
:1041160026F56DC327F547C028F548C029F52FECCD
:1041260015F00B0E0B6E260E0C6E5D0E0D6E0D2E23
:10413600FED70C2EFCD70B2EFAD70000000000018C
:10414600694B6A2B9ED7DD0E0501266F030E276F7E
:10415600520E176F650E186F730E196F650E1A6F74
:10416600740E1B6F1C6B170E286F050E296F7CECE7
:1041760011F000C0E3F001C0E4F0000E026E015041
:10418600025C02E10050000823E2070E05013C6FC5
:104196004C0E3D6F000E3E6F8CEC05F0C6EC10F039
:1041A600410E3C6F4C0E3D6F000E3E6F8CEC05F0E1
:1041B600B5EC05F00B0E0B6E260E0C6E5D0E0D6E3D
:1041C6000D2EFED70C2EFCD70B2EFAD700000000C2
:1041D6000501DD0E266F030E276F480E1D6F650E57
:1041E6001E6F6C0E1F6F700E206F216B1D0E286FD9
:1041F600050E296F7CEC11F000C0E3F001C0E4F07D
:10420600000E026E0150025C02E1005000080BE253
:10421600320E05013C6F460E3D6F000E3E6F8CEC74
:0C42260005F0AAEC05F034EF19F0FFD70A
:104DF80010EE1DF0410E006E010E016E7E0EF66E75
:0E4E0800480EF76E000EF86ECDEC0BF01200A7
:10423200000000000000000000000000000000007C
:10424200000000000000000000000000000000006C
:10425200000000000000000000000000000000005C
:10426200000000000000000000000000000000004C
:10427200000000000000000000000000000000003C
:10428200000000000000000000000000000000002C
:10429200000000000000000000000000000000001C
:1042A200000000000000000000000000000000000C
:1042B2000000000000000000424242000042424270
:1042C200844221000084422100E700000000E70050
:1042D200214284000021428401020408102040800F
:1042E2008040201008040201AA55AA55AA55AA55D1
:1042F200815A244242245A810058640404645800BA
:104302000C1222444422120C7E81A59191A5817E39
:104312007E8195A1A195817E20342AE1E12A342073
:1043220010F884828284F810985CB65F5FB65C985D
:1043320000000000000000000000009F00000000DC
:10434200000007000007000000247E24247E2400D1
:1043520000242A7F2A1200000043231008C4C2004E
:104362000076899562608000000009050300000064
:10437200000018244281000000008142241800003D
:104382000014087F081400000010107C10100000B8
:1043920000001090700000000010101010101000AB
:1043A2000000C0C00000000000402010080402000D
:1043B200007EA19189857E0000848281FF80800039
:1043C2000082C1A191898600004281898989760093
:1043D2000030282422FF2000008F898989897100FA
:1043E200007E9191919160000001E11109050300A5
:1043F20000768989898976000006898989493E0083
:104402000000006666000000000000AC6C000000C6
:104412000000081422410000002424242424240043
:104422000000412214080000000201B10906000048
:10443200000000000000000000FE21212121FE00FA
:1044420000FF898989897600007E8181818142000D
:1044520000FF818181423C0000FF898989818100BE
:1044620000FF090909010100007E81819191F2009A
:1044720000FF08080808FF00008181FF8181000019
:1044820000408081817F010000FF181824428100D2
:1044920000FF80808080800000FF02040402FF0091
:1044A20000FF04081020FF00007E818181817E00D0
:1044B20000FF090909090600007E8181A141BE00B1
:1044C20000FF0919294986000086898989897100B6
:1044D200000101FF01010000007F808080807F00D9
:1044E200003F408080403F00007F806060807F000E
:1044F20000C324181824C300000708F0F0080700BE
:1045020000C1A1918985830000FF81810000000024
:10451200001516FC161500000000008181FF000046
:10452200000402010204000000808080808080007C
:1045320000010204000000000020545454780000DE
:10454200007E4848483000000038444444200000BF
:1045520000304848487E0000003C4A4A4A0C0000AD
:1045620000107C1202040000000C5252523E000065
:10457200007E100808700000000000447D4000002A
:1045820000204040443D00000000FE205088000012
:10459200000082FE80800000007804180478000089
:1045A200007C0804047800000038444444380000C9
:1045B200007C14140800000000081414187C000089
:1045C200007C080404080000004854542400000041
:1045D20000043E4440200000003C4040207C00009B
:1045E200001C2040201C0000003C4030403C0000E9
:1045F200004428102844000000000C50503C0000E9
:10460200004464544C44000000000836410000009D
:10461200000000FF0000000000000041360800001A
:10462200000006090906000000103854101010009E
:104632003C4D73673D3E2020204C206D6178693DE2
:1046420031323220636172730D0A3C5265736574B4
:104652003E202052652D496E697420616666696349
:104662006865757273204D4158373231390D0A3CF5
:1046720054454D505F4F4E3E20202041666669638F
:104682006865206C612054656D702E20445331386A
:104692004232300D0A3C54454D505F4F46463E2053
:1046A20020456E6C65766520416666696368616760
:1046B2006520445331384232300D0A3C53706565EF
:1046C200643D3E20202056697465737365206465DD
:1046D20066696C656D656E74203A76616C6575729B
:1046E200206465203220E0203235300D0A3C4565D9
:1046F20070726F6D3D3E2020204D6573736167655A
:1047020020656E20656570726F6D2061766563202D
:10471200696E64696365203120E02031350D0A3C01
:10472200553B30343B30363B31343B30343B31390E
:104732003B3539233E20204D616A206465206C613F
:10474200205254430D0A3C44656D6F3E2020206187
:1047520066666963686520746F7573206C65732083
:104762006D6573736167657320656E2045455052B0
:094772004F4D205049430D0A008F
:10477B0020536F75726365203A205F3138463436AB
:10478B004B32325F746573745F4D61783731323100
:10479B00395F38784D6174726963653878385F5367
:1047AB004F46545F5350495F445331333031375F79
:1047BB00493243325F4C4D3333355F31383132320E
:1047CB00322E635F3138313232352E63200D0A00C1
:0247DB002000BC
:0647DD002053656320007B
:0247E3002000B4
:0547E5004D73673D006B
:1047EA000D0A68656C6C6F2C2069206765742079E6
:0947FA006F7572204D73672100F8
:0848030054454D505F4F4E007B
:09480B0054454D505F4F46460034
:0748140053706565643D006F
:08481B00456570726F6D3D00F0
:0548230044656D6F000B
:0648280052657365740087
:05482E0048656C7000FC
:104833002050726F6A6574203A2031384634364B03
:1048430032325F4D4158373231395F38785F4D61CD
:10485300745F3878385F535049315F536F667477AC
:104863005F4C4D3333355F4453313330375F493217
:0B48730043322E6D63707069720A0002
:10487E00274C00BF48003348007B47003C4900B23C
:0E488E004900BC4A00234A00EC4C00EA4D00F1
:04489C000000000018
:0448A0000000000014
:0448A4000000000010
:0248A8006400AA
:0448AA008C3D25001C
:0448AE000000000006
:0448B2000000000002
:0248B600000000
:0248B8000000FE
:0148BA0000FD
:0448BB0000000000F9
:1048BF00204469726563746F7279203A20433A5FBE
:1048CF004D696B726F435F4D657350726F6A65749C
:1048DF00735F4D696B726F435F31384634364B32BD
:1048EF00325F365F4D6174726978387838200D0AFF
:0148FF0000B8
:10490000496E6974204932433220285244303D5365
:10491000434C3229206574205244313D5344413286
:1049200020293430304B687A20706F7572205254D1
:0C4930004320445331333037200D0A007F
:10493C002036204D6F64756C6573204D61747269FF
:10494C006365203878382061766563204D4158378F
:10495C00313239202B2063617074657572204F578A
:0C496C005320445331384232300D0A0011
:10497800496E6974206574207465737420696E7457
:104988006572727570742054696D657231202032B9
:1049980030207820313030206D73656320736F6963
:0A49A800742032736563200D0A00CD
:1049B2002053616973697220756E206E6F7576651A
:1049C2006175204D73672061766563206C65207484
:1049D20065726D696E616C20766961203C4D73670A
:0949E2003D787878783E0D0A005A
:1049EB0041666669636865204D65737361676573BE
:1049FB00203020E0203135202073746F636B65739A
:104A0B0020656E20454550524F4D2064752050490E
:084A1B0043313846200D0A006A
:104A2300204D6573736167657320656E204545503E
:104A3300524F4D206176656320636465203A203CC4
:104A4300454550524F4D3D303E202E2E20E0203123
:054A530035200D0A00F2
:104A5800534F46542053504920205243333D436C12
:104A68006B202C5243353D446F75742020524330DF
:104A78003D4353202D3E204D4178373231393A0D90
:024A88000A0022
:104A8A00446973706C6179203C3031323334353685
:104A9A0037383941423E207375722036206D617471
:104AAA00726963657320387838204C656473200D09
:024ABA000A00F0
:104ABC00204D6F64652054656D70657261747572FC
:104ACC00652061766563203C54454D505F4F4E3EEA
:104ADC00206F75203C54454D505F4F46463E0D0AA5
:014AEC0000C9
:104AED000D0A4F4B2C2054656D7065722069732033
:104AFD004F4646210D0A5265746F757220617520FF
:0F4B0D00646973706C617920747874200D0A00EC
:104B1C00202020202020426F6E6E6520416E6E6535
:104B2C006520323031392E426F6E6E652053616EC6
:0E4B3C0074652E426967204269736F757300BD
:104B4A00525443204D414A20617520666F726D614F
:104B5A0074203A2020553B30343B30363B31343BCD
:0C4B6A0030343B31393B3539230D0A0053
:104B76004461746520267432202046696E202032F6
:104B86003031392F30312F30312030304830304DF0
:064B96003030533D200009
:104B9C00446174652026743120646562757420321A
:104BAC003031382F31322F32312031384835354DB4
:064BBC00353953203D00D5
:104BC2000D0A436C6F636B20696E697469616C6571
:104BD20020696E20203D20202E2E2E20204B687A28
:044BE200200D0A0098
:104BE60044617465202654322061752033312F319B
:104BF600322F31382032333A35393A3539203D2093
:014C060000AD
:104C0700526573657420416666696368657572737A
:104C1700204D61747269636520387838200D0A0069
:104C2700204D696B726F6320372E322E302031385A
:0A4C37004634364B3232200D0A00DD
:104C4100436C656172204D617472696365203678C9
:074C5100203878380D0A003D
:104C58000A0D4D6973652061206C2768657572655A
:074C680020525443203A00E2
:104C6F00436C656172204D6174726963652036789B
:074C7F00203878380D0A000F
:104C86002020456570726F6D204D736720616472D8
:064C960065737365200048
:104C9C000D0A4F4B2C2054656D7065722069732082
:064CAC004F4E210D0A002D
:104CB20054657374207265672E2044533138423232
:044CC200300D0A00A7
:104CC6000D0A4368616E67652053706565642054FC
:034CD6006F20004C
:104CD9002050726573656E746174696F6E203A2035
:034CE9000D0A00B1
:104CEC0020416C696D203D332E37565F6D696E69BE
:034CFC000D0A009E
:104CFF004E6577204453313330372044617465203B
:024D0F003A0068
:104D11000A0D205254432055706461746564200D5E
:024D21000A0086
:104D23004461746520267431204E6F77203D200046
:104D330030313233343536373839414243444546CE
:0F4D430046616D696C7920436F6465203A2000EA
:0F4D520020446966666572656E6365203D2000CA
:0E4D61004453313330372044617465203A00EA
:0D4D6F00446966666572656E6365203D00EF
:0D4D7C00303132333435363738394142009A
:0C4D8900204E65772054696D653A2000CB
:0B4D95002020736F6974203D3E200059
:0B4DA000436F6D70746575723D20005C
:0A4DAB00456570726F6D2023200033
:094DB500202020202020202000F5
:084DBE002054696D653A2000E4
:084DC60020204352433D200070
:074DCE00202020202020001E
:074DD5000D0A206D3D2000D6
:074DDC00204944313D200095
:074DE3002020202020200009
:054DEA00202020200044
:054DEF00B0432020008C
:044DF4003E3E20001F
:020000040030CA
:0D000100281E3CFF9980FF0FC00FE00F404C
:0200000400F00A
:100000005061676520576562203A207061756C66A3
:100010006A756A6F2E667265652E6672203A2020B8
:1000200020506171756573203230313820202020D6
:10003000415652494C202020200020202020202002
:1000400050696331384634364B323220204D696B6B
:10005000726F432050726F20372E312E30202020B7
:100060003136204D65736720656E20454550524FEF
:100070004D206465203634206361726163742E0004
:100080004A6575782064652063617220204153437E
:100090004949646520203020E0203132372020207B
:1000A0004142434445464748494A4B4C4D4E4F50C8
:1000B0005152535455565758595A2061626364003F
:1000C00065666768696A6B6C6D6E6F707172737468
:1000D000757778797A23242B2D5F5B5D26B03D20E0
:1000E00020426F6E6E6520416E6E65652032303144
:1000F0003820002020202020202020202020200028
:1001000031382020202020202020202020202000E6
:100110005241532000202020202020202020200099
:100120005A65726F002020202020202020202000EF
:1001300057616C6F75002020202020202020200097
:100140005269656E002020202020202020202000E1
:10015000456D707479002020202020202020200070
:100160004C656572200020202020202020202000C7
:100170005269656E200020202020202020202000B1
:100180007669646500202020202020202020200087
:100190005269656E00202020202020202020200091
:1001A0004E49422000202020202020202020200016
:1001B000456D707479002020202020202020200010
:1001C000456D707479002020202020202020200000
:1001D000456D7074790020202020202020202000F0
:1001E000456D7074790020202020202020202000E0
:1001F000456D7074790020202020202020202000D0
:10020000456D7074790020202020202020202000BF
:10021000456D7074790020202020202020202000AF
:10022000456D70747900202020202020202020009F
:10023000456D70747900202020202020202020008F
:10024000456D70747900202020202020202020007F
:10025000456D70747900202020202020202020006F
:10026000456D70747900202020202020202020005F
:10027000456D70747900202020202020202020004F
:10028000456D70747900202020202020202020003F
:10029000456D70747900202020202020202020002F
:1002A000456D70747900202020202020202020001F
:1002B000456D70747900202020202020202020000F
:1002C000456D7074790020202020202020202000FF
:1002D000456D7074790020202020202020202000EF
:1002E000456D7074790020202020202020202000DF
:1002F000456D7074790020202020202020202000CF
:10030000456D7074790020202020202020202000BE
:10031000456D7074790020202020202020202000AE
:10032000456D70747900202020202020202020009E
:10033000456D70747900202020202020202020008E
:10034000456D70747900202020202020202020007E
:10035000456D70747900202020202020202020006E
:10036000456D70747900202020202020202020005E
:10037000456D70747900202020202020202020004E
:10038000456D70747900202020202020202020003E
:10039000456D70747900202020202020202020002E
:1003A000456D70747900202020202020202020001E
:1003B000456D70747900202020202020202020000E
:1003C000456D7074790020202020202020202000FE
:1003D000456D7074790020202020202020202000EE
:1003E000456D7074790020202020202020202000DE
:1003F000456D7074790020202020202020202000CE
:00000001FF
